:1000000033C0000044C0000042C0000040C00000F7
:100010003EC000003CC000003AC0000038C00000F4
:1000200036C0000034C0000032C0000030C0000004
:100030002EC000002CC000002AC0000028C0000014
:1000400026C0000024C0000022C0000020C0000024
:100050001EC000001CC000001AC0000018C0000034
:1000600016C0000014C0000011241FBECFEFD8E05E
:10007000DEBFCDBF12E0A0E0B1E0E6EAFEE002C0E4
:1000800005900D92A633B107D9F737D00AC7B8CF7C
:1000900060E070E088EC92E467D021E030E04497C3
:1000A00011F020E030E0C901089560E070E083EED7
:1000B00093E414D121E030E0892B11F020E030E00E
:1000C000C901089560E070E088E694E407D121E07A
:1000D00030E0C29711F020E030E0C901089560E0FF
:1000E00070E68FEA94E4FAD021E030E0843691059E
:1000F00011F020E030E0C90108950CD024E030E098
:1001000040E051E060E171E088E191E0F0D080E012
:1001100090E008951092C5008CE08093C400E0EC5C
:10012000F0E080818260808388E18093C10086E076
:100130008093C20008959091C00095FFFCCF8093FA
:10014000C60008951F93CF93DF93EC0110E0FE01EA
:10015000E10FF11D8081882319F0EDDF1F5FF7CFDC
:10016000DF91CF911F91089520E030E040EA50E404
:10017000D0D181D336D2CB0108958F929F92AF9286
:10018000BF92CF92DF92EF92FF920F931F93CF9384
:10019000DF934B015C01EA0169016881798188275D
:1001A00077FD8095982F50D29B01AC01C501B40119
:1001B000ACD187FF05C06A817B818C819D8181C024
:1001C00086E08C9D80018D9D100D11240650110933
:1001D0000C0F1D1FF80160817181882777FD8095C4
:1001E000982F32D29B01AC01C501B401DDD21816A3
:1001F0000CF462C08E0180E090E0F1E0CF1AD108EB
:100200009C012F5F3F4F79018C159D0584F4F80107
:1002100066817781882777FD8095982F15D20A5FB0
:100220001F4FA5019401C0D218160CF043C086E000
:100230008E9DF0018F9DF00D11248E010E0F1F1F5A
:100240003697EC0FFD1FC081D181C280D380E4803E
:10025000F580BE01882777FD8095982FF5D19B0109
:10026000AC01C501B401ECD04B015C01A7019601C2
:10027000F8016281738184819581E2D09B01AC0198
:10028000C501B40195D24B015C01F8016081718117
:100290006C1B7D0B882777FD8095982FD5D19B010E
:1002A000AC01C501B40135D19B01AC01C701B60158
:1002B000C8D007C0C701A4CFF801628173818481CF
:1002C0009581DF91CF911F910F91FF90EF90DF907B
:1002D000CF90BF90AF909F908F90089526E030E030
:1002E00048E551E04ADFC7D27CD1CB0108953F9267
:1002F0004F925F926F927F928F929F92AF92BF9236
:10030000CF92DF92EF92FF920F931F93CF93DF93E1
:10031000CDB7DEB7C258D1090FB6F894DEBF0FBE15
:10032000CDBF182F092F562E472E79018CE791E06B
:10033000CF57DF4F4883C158D040CE57DF4F588347
:10034000C258D040FFDEFF92EF920F931F9384EAD2
:1003500091E09F938F931F9280E48F938E010F5BA8
:100360001F4F1F930F93D0D2C801ECDECF57DF4F42
:100370004881C158D040042FCE57DF4F5881C25812
:10038000D040152F0FB6F894DEBF0FBECDBFC12CE5
:10039000D12C86EC882E81E0982E90E4392EDE0157
:1003A00011965D01CE14DF0454F5D8011296ED913B
:1003B000FC91139709953C01F80181818F9380810D
:1003C0008F934F925F929F928F921F923F92BF9214
:1003D000AF929AD2C501B6DE0FB6F894DEBF0FBE5B
:1003E000CDBF672819F48BEE91E0ACDE8AE192E094
:1003F000A9DE9FEFC91AD90A0C5F1F4FD3CF87E23E
:1004000092E0A0DE84EC91E09DDE84E094DECE57A5
:10041000DF4F0FB6F894DEBF0FBECDBFDF91CF9197
:100420001F910F91FF90EF90DF90CF90BF90AF9012
:100430009F908F907F906F905F904F903F90089526
:100440005058BB27AA270ED075C166D130F06BD1AA
:1004500020F031F49F3F11F41EF45BC10EF4E095DF
:10046000E7FB51C1E92F77D180F3BA176207730711
:100470008407950718F071F49EF58FC10EF4E0958E
:100480000B2EBA2FA02D0B01B90190010C01CA014E
:10049000A0011124FF27591B99F0593F50F4503EF9
:1004A00068F11A16F040A22F232F342F4427585FEB
:1004B000F3CF469537952795A795F0405395C9F703
:1004C0007EF41F16BA0B620B730B840BBAF09150BB
:1004D000A1F0FF0FBB1F661F771F881FC2F70EC05A
:1004E000BA0F621F731F841F48F48795779567952D
:1004F000B795F7959E3F08F0B3CF9395880F08F016
:100500009927EE0F979587950895D9D008F481E043
:1005100008950CD00FC107D140F0FED030F021F487
:100520005F3F19F0F0C0511139C1F3C014D198F3F5
:100530009923C9F35523B1F3951B550BBB27AA2764
:1005400062177307840738F09F5F5F4F220F331FD6
:10055000441FAA1FA9F333D00E2E3AF0E0E830D0A2
:1005600091505040E695001CCAF729D0FE2F27D0A5
:10057000660F771F881FBB1F261737074807AB0773
:10058000B0E809F0BB0B802DBF01FF2793585F4FE8
:100590002AF09E3F510568F0B6C000C15F3FECF302
:1005A000983EDCF3869577956795B795F7959F5FAD
:1005B000C9F7880F911D9695879597F90895E1E001
:1005C000660F771F881FBB1F621773078407BA0760
:1005D00020F0621B730B840BBA0BEE1F88F7E095BB
:1005E000089504D06894B111D9C00895BCD088F0A2
:1005F0009F5790F0B92F9927B751A0F0D1F0660F0F
:10060000771F881F991F1AF0BA95C9F712C0B13029
:1006100081F0C3D0B1E00895C0C0672F782F88273C
:10062000B85F39F0B93FCCF3869577956795B39568
:10063000D9F73EF490958095709561957F4F8F4FD7
:100640009F4F0895E89409C097FB3EF490958095DC
:10065000709561957F4F8F4F9F4F9923A9F0F92F88
:1006600096E9BB279395F695879577956795B79506
:10067000F111F8CFFAF4BB0F11F460FF1BC06F5FEC
:100680007F4F8F4F9F4F16C0882311F096E911C0FE
:10069000772321F09EE8872F762F05C0662371F01F
:1006A00096E8862F70E060E02AF09A95660F771F33
:1006B000881FDAF7880F9695879597F90895990F0F
:1006C0000008550FAA0BE0E8FEEF16161706E8071C
:1006D000F907C0F012161306E407F50798F0621B3D
:1006E000730B840B950B39F40A2661F0232B242B12
:1006F000252B21F408950A2609F4A140A6958FEF31
:10070000811D811D089597F99F6780E870E060E082
:1007100008959FEF80EC089500240A94161617069A
:1007200018060906089500240A94121613061406E2
:1007300005060895092E0394000C11F4882352F045
:10074000BB0F40F4BF2B11F460FF04C06F5F7F4FFD
:100750008F4F9F4F089557FD9058440F551F59F0E4
:100760005F3F71F04795880F97FB991F61F09F3F9E
:1007700079F087950895121613061406551FF2CFC7
:100780004695F1DF08C0161617061806991FF1CF17
:1007900086957105610508940895E894BB2766273E
:1007A0007727CB0197F908958ADF08F48FEF089532
:1007B0000BD0C0CFB1DF28F0B6DF18F0952309F0D9
:1007C000A2CFA7CF1124EACFC6DFA0F3959FD1F324
:1007D000950F50E0551F629FF001729FBB27F00DEF
:1007E000B11D639FAA27F00DB11DAA1F649F662744
:1007F000B00DA11D661F829F2227B00DA11D621F93
:10080000739FB00DA11D621F839FA00D611D221F4C
:10081000749F3327A00D611D231F849F600D211D30
:10082000822F762F6A2F11249F5750408AF0E1F0D3
:1008300088234AF0EE0FFF1FBB1F661F771F881F1C
:1008400091505040A9F79E3F510570F05CCFA6CF64
:100850005F3FECF3983EDCF3869577956795B79507
:10086000F795E7959F5FC1F7FE2B880F911D969531
:10087000879597F9089577DFE0F09E37D8F096399D
:10088000B8F49E3848F4672F782F8827985FF9CFFF
:1008900086957795679593959539D0F3B62FB17076
:1008A0006B0F711D811D20F4879577956795939542
:1008B00002C01CC073CF882371F4772321F09850B5
:1008C000872B762F07C0662311F499270DC090510E
:1008D000862B70E060E02AF09A95660F771F881FDC
:1008E000DAF7880F9695879597F908959F3F31F02D
:1008F000915020F4879577956795B795880F911D4E
:100900009695879597F90895AEE0B0E0E9E8F4E0B0
:100910009FC20D891E898F89988D26E02C831A83AA
:10092000098397FF02C080E090E801979E838D8342
:10093000AE01455E5F4F698D7A8DCE01019611D073
:100940004D815E8157FD0AC02F81388542175307BC
:100950000CF49A01F801E20FF31F10822E96E4E0E6
:1009600093C2ACE0B0E0E6EBF4E064C27C016B0162
:100970008A01FC0117821682838181FFB0C1CE01FA
:1009800001964C01F7019381F60193FD859193FF48
:1009900081916F01882309F49EC1853239F493FD5A
:1009A000859193FF81916F01853221F4B70190E029
:1009B000B1D1E8CF512C312C20E02032A0F48B3281
:1009C00069F030F4803259F0833269F420612CC030
:1009D0008D3239F0803339F4216026C022602460E2
:1009E00023C0286021C027FD27C030ED380F3A30E2
:1009F00078F426FF06C0FAE05F9E300D1124532ED6
:100A000013C08AE0389E300D1124332E20620CC0B2
:100A10008E3221F426FD5FC1206406C08C3611F4AD
:100A2000206802C0883641F4F60193FD859193FF5A
:100A300081916F018111C1CF982F9F7D9554933083
:100A400028F40C5F1F4FFFE3F9830DC0833631F0AC
:100A5000833771F0833509F057C021C0F8018081D8
:100A600089830E5F1F4F44244394512C540114C0BA
:100A70003801F2E06F0E711CF801A080B18026FFF2
:100A800003C0652D70E002C06FEF7FEFC5012C87BA
:100A900036D12C0183012C852F77222E16C03801E8
:100AA000F2E06F0E711CF801A080B18026FF03C038
:100AB000652D70E002C06FEF7FEFC5012C8714D168
:100AC0002C012C852068222E830123FC19C0832D44
:100AD00090E048165906A0F4B70180E290E01AD1E0
:100AE0003A94F5CFF50127FC859127FE81915F01AE
:100AF000B70190E00FD131103A94F1E04F1A51084C
:100B00004114510479F7DEC0843611F0893631F58D
:100B1000F80127FF07C060817181828193810C5F9A
:100B20001F4F08C060817181882777FD8095982FBD
:100B30000E5F1F4F2F76B22E97FF09C090958095BC
:100B4000709561957F4F8F4F9F4F2068B22E2AE09E
:100B500030E0A40111D1A82EA81843C0853729F48C
:100B60002F7EB22E2AE030E025C0F22FF97FBF2E73
:100B70008F36C1F018F4883579F0ADC0803719F0A0
:100B8000883721F0A8C02F2F2061B22EB4FE0DC0EF
:100B90008B2D8460B82E09C024FF0AC09F2F966059
:100BA000B92E06C028E030E005C020E130E002C0E8
:100BB00020E132E0F801B7FE07C0608171818281D7
:100BC00093810C5F1F4F06C06081718180E090E0CF
:100BD0000E5F1F4FA401D0D0A82EA818FB2DFF77C1
:100BE000BF2EB6FE0BC02B2D2E7FA51450F4B4FEE5
:100BF0000AC0B2FC08C02B2D2E7E05C07A2C2B2DEE
:100C000003C07A2C01C0752C24FF0DC0FE01EA0D33
:100C1000F11D8081803311F4297E09C022FF06C0B6
:100C20007394739404C0822F867809F0739423FD23
:100C300012C020FF06C05A2C731418F4530C571816
:100C4000732C731460F4B70180E290E02C8762D0BB
:100C500073942C85F6CF731410F4371801C0312C1F
:100C600024FF11C0B70180E390E02C8753D02C857E
:100C700022FF16C021FF03C088E590E002C088E78C
:100C800090E0B7010CC0822F867851F021FD02C0A0
:100C900080E201C08BE227FD8DE2B70190E03AD0FF
:100CA000A51430F4B70180E390E034D05A94F8CF23
:100CB000AA94F401EA0DF11D8081B70190E02AD0D9
:100CC000A110F6CF332009F45DCEB70180E290E0A9
:100CD00021D03A94F7CFF7018681978102C08FEF38
:100CE0009FEF2C96E2E1C2C0FC010590615070407C
:100CF0000110D8F7809590958E0F9F1F0895FC01E5
:100D00006150704001900110D8F7809590958E0F3A
:100D10009F1F08950F931F93CF93DF93182F092FD1
:100D2000EB018B8181FD03C08FEF9FEF20C082FF1D
:100D300010C04E815F812C813D81421753077CF4A6
:100D4000E881F9819F012F5F3F4F3983288310830A
:100D500006C0E885F985812F0995892B29F72E8111
:100D60003F812F5F3F4F3F832E83812F902FDF9155
:100D7000CF911F910F910895FA01AA27283051F1C0
:100D8000203181F1E8946F936E7F6E5F7F4F8F4FBC
:100D90009F4FAF4FB1E03ED0B4E03CD0670F781F1B
:100DA000891F9A1FA11D680F791F8A1F911DA11D00
:100DB0006A0F711D811D911DA11D20D009F4689439
:100DC0003F912AE0269F11243019305D3193DEF6E1
:100DD000CF010895462F4770405D4193B3E00FD097
:100DE000C9F7F6CF462F4F70405D4A3318F0495D82
:100DF00031FD4052419302D0A9F7EACFB4E0A69565
:100E00009795879577956795BA95C9F70097610586
:100E1000710508959B01AC010A2E069457954795DC
:100E200037952795BA95C9F7620F731F841F951FD1
:100E3000A01D08952F923F924F925F926F927F92E2
:100E40008F929F92AF92BF92CF92DF92EF92FF92DA
:100E50000F931F93CF93DF93CDB7DEB7CA1BDB0B86
:100E60000FB6F894DEBF0FBECDBF09942A8839882B
:100E700048885F846E847D848C849B84AA84B98432
:100E8000C884DF80EE80FD800C811B81AA81B9813E
:100E9000CE0FD11D0FB6F894DEBF0FBECDBFED0152
:060EA0000895F894FFCF55
:100EA6001F0148002B0155003901620048016F00FF
:100EB60073656E736F7273006C616D62646100744A
:100EC600657374546F54656D70490074657374541A
:100ED6006F54656D704F30430074657374546F546E
:100EE600656D704F3530430074657374546F546587
:100EF6006D704F3130304300C7FF000048C2C60155
:100F0600000000007B050000C842D80800004843E6
:100F1600E70B00009643B20E0000C8433C3F786DD5
:100F26006C2076657273696F6E3D22312E302220F9
:100F3600656E636F64696E673D225554462D38228F
:100F46003F3E0A003C746573747375697465206E60
:100F5600616D653D222573222074657374733D228D
:100F66002564223E0A003C746573746361736520D0
:100F7600636C6173736E616D653D22257322206E0D
:100F8600616D653D222573223E0A003C6661696CEF
:100F960075726520747970653D226661696C75723B
:100FA60065223E54657374206661696C65643C2FE6
:100FB6006661696C7572653E0A003C2F74657374D0
:100FC600636173653E0A003C2F74657374737569BB
:060FD60074653E0A0000F4
:00000001FF
